:1000000016C030C02FC02EC02DC02CC02BC02AC09F
:1000100029C028C027C026C025C024C023C022C0B4
:1000200021C020C01FC00C12120C000000001124BF
:100030001FBECFE5D4E0DEBFCDBF10E0A0E6B0E04C
:10004000ECEDF4E002C005900D92AE3AB107D9F79D
:1000500010E0AEEAB0E001C01D92AE3AB107E1F7A0
:100060001DD03AC2CDCF089580E886B985E886B91B
:1000700017B8089597B1907E97B987B9369A349B8F
:10008000FECF3498369A349BFECF349894B185B124
:10009000382F20E0290F311DC90108952F923F927A
:1000A0004F925F926F927F928F929F92AF92BF9288
:1000B000CF92DF92EF92FF920F931F93DF93CF9334
:1000C000CDB7DEB7C457D0400FB6F894DEBF0FBE31
:1000D000CDBFDE011B96E0E6F0E08CE001900D92D2
:1000E0008150E1F7DE015796ECE6F0E08CE00190FC
:1000F0000D928150E1F7DE019396E8E7F0E08DE0A4
:1001000001900D928150E1F7DE01D096E5E8F0E034
:100110008DE001900D928150E1F7DE01A75ABF4FAB
:10012000E2E9F0E08EE001900D928150E1F7DE010E
:10013000A959BF4FE0EAF0E08EE001900D928150A6
:10014000E1F78CE03BD190DFEE24FF2400E010E0EB
:100150002E010894411C511C36E0632E712C6C0E4C
:100160007D1E2DE3822E912C8C0E9D1E9BE4A92ECC
:10017000B12CAC0EBD1E8BE0282E312C2C0E3D1E5A
:1001800006C080E077DFE80EF91E0F5F1F4F0931D0
:100190001105B8F3C70169E170E077D1CB018C5943
:1001A000914063E070E085D16B01EE24FF2400E014
:1001B00010E081E05FDFE80EF91E0F5F1F4F09318D
:1001C0001105B9F7C70169E170E05FD1CB018F5923
:1001D000914063E070E06DD18B0187EFC8168FEF1F
:1001E000D8061CF4C401B1010DC0C60101970997DE
:1001F00028F0C401BE016D5D7F4F04C0C401BE0183
:10020000675A7F4F0CD1EFEF073F1E072CF4C50153
:10021000BE01695E7F4F0DC0C8010197099728F0A4
:10022000C501BE01605D7F4F04C0C501BE016959B3
:100230007F4FF5D0C601B2014AE050E0F7D0C801C7
:10024000B3014AE050E0F2D080E46ED006E210E064
:10025000F801849171D00F5F1F4FF0E00E321F073D
:10026000B9F77CD0C40192D0C20190D08EE060E09A
:100270006BD080E079D083E477D080E061E064D017
:10028000C50184D0C30182D08EE061E05DD080E002
:100290006BD083E469D0EE24FF2400E010E077CF38
:1002A000282F662311F0C49A01C0C498C59887B35B
:1002B0008F6087BB98B3907F822F82958F70892B38
:1002C00088BBC69A00C0C6982F70292B28BBC69A37
:1002D00000C0C6989F6098BB0895C498C59A87B31C
:1002E000807F87BBC69A00C086B3C69800C0C69AF6
:1002F00000C096B3C69883FDF0CF82E090E00197EE
:10030000F1F7C498C59A87B3807F87BBC69A00C0AF
:1003100096B3C69800C0C69A00C086B38F709295F7
:10032000907FC698892B08951F93182FD6DF812FB1
:1003300060E0B6DF1F9108951F93182FCEDF812F45
:1003400061E0AEDF1F910895662311F4805801C06B
:100350008054EADF0895C1DF90E0089581E0E4DF92
:10036000089582E0E1DF08951F93182FB6DF1A3059
:1003700041F4803410F080E001C080E48058D4DF84
:1003800003C0812F61E08CDF1F910895CF93DF932D
:10039000EC0101C0E9DF89918823E1F7DF91CF917A
:1003A0000895CF93DF93EC0101C0DEDFFE012196BB
:1003B00084918823D1F7DF91CF9108951F93182F4F
:1003C00087B38F6787BB80E89EE30197F1F7C19AF7
:1003D000C09AC69A00C0C69880E893E10197F1F7E9
:1003E000C69A00C0C69880E490E0FC013197F1F70E
:1003F000C69A00C0C698FC013197F1F7C098C69A1A
:1004000000C0C6980197F1F788E28EDF88E08CDFA4
:10041000A5DF86E089DF812F87DF1F910895FB012B
:10042000DC0101900D920020E1F70895FB019F018E
:10043000E8944230BCF04532ACF44A3029F497FBE2
:100440001EF4909581959F4F642F77271ED0805D75
:100450008A330CF0895D8193CB010097A9F716F4DC
:100460005DE251931082C90100C0DC01FC01672FDD
:1004700071917723E1F7329704C07C916D9370837B
:100480006291AE17BF07C8F30895AA1BBB1B51E1C9
:1004900007C0AA1FBB1FA617B70710F0A61BB70BF4
:1004A000881F991F5A95A9F780959095BC01CD0199
:1004B000089597FB092E07260AD077FD04D0E5DFC3
:1004C00006D000201AF4709561957F4F0895F6F7D5
:0C04D000909581959F4F0895F894FFCF00
:1004DC00496E6E656E3A20202020200041757373A2
:1004EC00656E3A2020202000496E6E656E3A202001
:1004FC00202020200041757373656E3A2020202047
:10050C002000496E6E656E3A2020202020202000AD
:0E051C0041757373656E3A2020202020200068
:00000001FF
